:020000040800F2
:10000000600F0020ED01000829130008A50B00086F
:100010002513000855030008891B00080000000094
:10002000000000000000000000000000F1190008BE
:1000300059030008000000002B1300080502000807
:10004000070200080702000807020008070200086C
:10005000070200080702000807020008070200085C
:10006000070200080702000807020008070200084C
:10007000070200080702000807020008070200083C
:10008000070200080702000807020008070200082C
:10009000070200080702000807020008070200081C
:1000A000070200080702000807020008070200080C
:1000B00007020008070200080702000807020008FC
:1000C00007020008070200080702000807020008EC
:1000D00007020008070200080702000807020008DC
:1000E00007020008070200080702000807020008CC
:1000F00007020008070200080702000807020008BC
:1001000007020008070200080702000807020008AB
:10011000070200080702000807020008070200089B
:10012000070200080702000807020008070200088B
:10013000070200080702000807020008070200087B
:10014000070200080702000807020008070200086B
:10015000070200080702000807020008070200085B
:10016000070200080702000807020008070200084B
:10017000070200080702000800000000000000005D
:10018000070200080702000807020008070200082B
:10019000070200080702000800000000070200082C
:1001A000070200080702000800000000000000002D
:1001B000070200080000000000000000070200081D
:1001C00007020008070200080702000807020008EB
:1001D0000702000807020008DFF80CD000F0A8F8BA
:1001E0000048004701220008600F002006488047B1
:1001F00006480047FEE7FEE7FEE7FEE7FEE7FEE70C
:10020000FEE7FEE7FEE7FEE76D1B0008D9010008E8
:100210002DE9F05F0546002092469B46884606463B
:10022000814640241BE0284641464746224600F0CE
:100230006EF853465A46C01A914110D311461846DB
:10024000224600F055F82D1A67EB01084F4622466A
:100250000120002100F04CF817EB00094E41201E50
:10026000A4F10104DFDC484631462A464346BDE896
:10027000F09F10B5431A934209D28318881803E0FF
:1002800010F8011D03F8011D521EF9D210BD40EAFD
:1002900001039B0703D009E008C9121F08C0042A04
:1002A000FAD203E011F8013B00F8013B521EF9D2EB
:1002B00010BDD2B201E000F8012B491EFBD27047FD
:1002C0000022F6E710B513460A4604461946FFF722
:1002D000F0FF204610BD30B504460020034600E084
:1002E0005B1C934203D2E05CCD5C401BF8D030BD78
:1002F000202A04DB203A00FA02F1002070479140E6
:10030000C2F1200320FA03F3194390407047202ADA
:1003100004DB203A21FA02F00021704721FA02F3AF
:10032000D040C2F1200291400843194670470000B6
:10033000064C074D06E0E06840F0010394E8070032
:1003400098471034AC42F6D3FFF74AFFE023000889
:100350000024000800BFFEE77047704710B5002278
:1003600001B909E0012901D10A0205E0022901D100
:100370000A0201E04FF440720E4B1B6823F44073F5
:100380000C4C236023461B681343236023461B68E1
:1003900023F07803236023461B68022444EAC00448
:1003A0002343044C236023461B6843F480332360BB
:1003B00010BD0000103C02401C48006800F40070B2
:1003C000B0B11A48006820F400701849086000BFF6
:1003D0000846006840F4006008600846006820F4A1
:1003E0000060086000BF0846006840F400700860C4
:1003F0000E48006800F48060B0B10C48006820F43A
:1004000080600A49086000BF0846006840F48050D8
:1004100008600846006820F48050086000BF084665
:10042000006840F48060086070470000003C0240B3
:100430000A4A126822F44072084B1A601A4612687F
:1004400042F004021A601A4612684FF4803343EAFD
:1004500000231A43014B1A6070470000103C024011
:10046000074A126822F44072054B1A601A46126855
:100470001A601A46126842F001021A600170704751
:10048000103C024010B50D49096821F440710B4C35
:1004900021602146096841F44071216021460968C4
:1004A00041F001012160026000BF00BF00BFBFF347
:1004B0006F8F00BF00BF00BF436010BD103C024003
:1004C000084A126822F44072064B1A601A461268F3
:1004D00042F480721A601A46126842F001021A60F1
:1004E00001807047103C0240084A126822F44072B2
:1004F000064B1A601A46126842F400721A601A46D5
:10050000126842F001021A6001607047103C02401C
:100510002A48006800F0100040B12948C06940F046
:1005200010002749C861102024490860234800684A
:1005300000F0200040B12248C06940F00800204986
:10054000C86120201D4908601C48006800F0400078
:1005500040B11B48C06940F004001949C8614020FF
:10056000164908601548006800F0800040B1144842
:10057000C06940F002001249C86180200F4908603C
:100580000E48006800F4807048B10D48C06940F022
:1005900001000B49C8614FF48070084908600748A2
:1005A000006800F0020040B10548C06940F020003A
:1005B0000349C86102200149086070470C3C0240B1
:1005C0003C0B002070B50446002500201449C8618A
:1005D00000F0E2FA054609E0601C38B124B100F0F1
:1005E000DBFA401BA04201D9032070BD0D48006812
:1005F00000F480300028EFD10A48006800F00100C4
:1006000010B10120074908600648006800F4F9703D
:1006100018B1FFF77DFF0120E7E70020E5E70000C4
:100620003C0B00200C3C02402DE9F0430B4620F02F
:10063000030600EB020C0CF1030C2CF00307002561
:10064000314635E00C68814207D300EB020C8C4543
:1006500003D9AC466D1C03F80C4001F1010C844534
:1006600009D300EB0208E04505D9C4F30729AC46DD
:100670006D1C03F80C9001F1020C844509D300EBCA
:100680000208E04505D9C4F30749AC466D1C03F8E0
:100690000C9001F1030C844509D300EB0208E045FE
:1006A00005D94FEA1469AC466D1C03F80C90091D7E
:1006B000B942C7D3BDE8F0832DE9F04103460C46AB
:1006C00023F003079818C01C20F0030C00263946BD
:1006D0003FE00D6899420CD39818884209D93046FA
:1006E000761C205C05F0FF08404502D00020BDE8E4
:1006F000F081481C98420CD303EB0208804508D9CE
:100700003046761C205CC5F30728404501D0002008
:10071000EDE7881C98420CD303EB0208804508D90A
:100720003046761C205CC5F30748404501D00020C8
:10073000DDE7C81C98420BD303EB0208804507D9BC
:100740003046761C205CB0EB156F01D00020CEE760
:10075000091D6145BDD30120C9E700002DE9F05F07
:1007600007468946144623E0384600F095F80646C9
:10077000304600F0F5F88346304600F0D7F8804662
:10078000A7EB080AABEB0A05A54200D925460A48A3
:10079000805D28B9384600F053F801200649885595
:1007A0002A464946384600F061F82F44A944641BA4
:1007B000002CD9D1BDE8F09F000000202DE9F041C8
:1007C00006460F4614461EE0C6F30A08C8F5006543
:1007D000A54200D925462A460D49384600F078FE44
:1007E0002A460B493046FFF7B9FF2A4608493046EA
:1007F000FFF762FF20B92A46314606A001F0C6F98C
:100800002F442E44641B002CDED1BDE8F081000093
:10081000280000202A2A2A205665726966792066F7
:100820006C617368206661696C6564206174202561
:100830003038582C2025642062797465730D0A00C5
:1008400038B504460020009007490860022008617E
:10085000204600F021F8044988600120C8606946FC
:10086000014800F0D3F838BD280800202DE9F041F8
:1008700005460E461746B046002408E058F804CB5B
:10088000291962460023022000F020F9241DBC42F1
:10089000F4D3BDE8F0810000014600201C4A9142DB
:1008A00003D2B1F1006F00D330E01A4A914204D272
:1008B000174A914201D3012028E0174A914204D2FD
:1008C000144A914201D3022020E0144A914204D2FA
:1008D000114A914201D3032018E0114A914204D2F7
:1008E0000E4A914201D3042010E00E4A914204D2F4
:1008F0000B4A914201D3052008E00B4A914204D2F1
:10090000084A914201D3062000E00720704700000A
:10091000004000080080000800C000080000010836
:10092000000002080000040800000608014600203C
:1009300029B1012903D0022901D0032904D10A4693
:10094000920302F1006007E0042901D1034803E0AB
:100950004A1F520402F100607047000000000108C5
:100960000146002029B1012903D0022901D0032921
:1009700002D14FF4804005E0042901D1880301E051
:100980004FF40030704700002DE9F05F81460E46BD
:1009900014461F464FF0000A002530E0207830B999
:1009A000316801EB09000122174900F091FD207820
:1009B000C0F1080000F0FF08781B404502DA781B00
:1009C00000F0FF08012000FA08F0401E1FFA80FB2B
:1009D00021780D480078084100EA0B00A84040EA61
:1009E0000A0A2078404420702078082804D1306812
:1009F000401C30600020207005EB0800C5B2BD42ED
:100A0000CCDB5046BDE8F09F100000202DE9F041FE
:100A100004460E460127002500BF2548007E012818
:100A200002D10220BDE8F08101202149087600BFF3
:100A30004CF25030FFF7C6FD0746002F31D1401E63
:100A40003060206801280FD1207C6168FFF7F0FC3E
:100A50004CF25030FFF7B6FD07461648006820F00C
:100A60000400144908601AE0A56812E0217C2846B9
:100A7000FFF774FC4CF25030FFF7A4FD07460D4819
:100A8000006820F07A000B4908600FB1356005E07E
:100A90006D1CD4E902100844A842E7D800BFFFF754
:100AA0008BFC00BF00200249087600BF3846B9E73A
:100AB0003C0B0020103C02400348006840F000401E
:100AC0000149086000207047103C02402DE9F041C8
:100AD00006460F4614461D464FF0010800BF1F484A
:100AE000007E012802D10220BDE8F08101201B49CF
:100AF000087600BF4CF25030FFF764FD8046B8F135
:100B0000000F23D126B9E1B23846FFF7A9FC12E065
:100B1000012E04D1A1B23846FFF7D2FC0BE0022E21
:100B200004D121463846FFF7DFFC04E022462B467D
:100B30003846FFF7A7FC4CF25030FFF743FD8046E4
:100B40000748006820F001000549086000BF002048
:100B50000249087600BF4046C6E700003C0B002073
:100B6000103C024000200949096801F0004159B1D8
:100B70000749064A0C3A11600649116003490968A1
:100B800001F0004101B1012070470000103C02401B
:100B900023016745AB89EFCD01480068704700002D
:100BA0001400002000BFFEE7044672B64FF0E020BC
:100BB000006920F003004FF0E0210861206880F315
:100BC000088800BF6068804702E002A000F0DEFFF6
:100BD000FBE700002E00000008B505490968014345
:100BE000034A1160114609680140009100BF08BD29
:100BF0003038024008B5054909680143034A1160CD
:100C0000114609680140009100BF08BD4438024008
:100C1000F0B502460B4600240021186890FAA0F0B7
:100C2000B0FA80F494E00125A540186800EA0501B7
:100C300000297DD05868012802D05868022826D1A2
:100C40009868956891FAA1F6B6FA86F677000326B9
:100C5000BE40B54391FAA1F6B6FA86F6760000FAE0
:100C600006F63543956000BFD868556891FAA1F63D
:100C7000B6FA86F70126BE40B54391FAA1F6B6FA58
:100C800086F600FA06F63543556000BF00BF1869C6
:100C9000D56891FAA1F6B6FA86F677000326BE402B
:100CA000B54391FAA1F6B6FA86F6760000FA06F692
:100CB0003543D56000BF5868022831D191FAA1F0C0
:100CC000B0FA80F0082814D25869156A91FAA1F692
:100CD000B6FA86F6B7000F26BE40B54391FAA1F6E4
:100CE000B6FA86F6B60000FA06F63543156200BF7E
:100CF00016E05869556A0E0A96FAA6F6B6FA86F60E
:100D0000B7000F26BE40B5430E0A96FAA6F6B6FA0D
:100D100086F6B60000FA06F63543556200BF00BFFE
:100D20005868156891FAA1F6B6FA86F6770000E0E1
:100D30000DE00326BE40B54391FAA1F6B6FA86F659
:100D4000760000FA06F63543156000BF00BF641C4C
:100D50001868E04000287FF466AFF0BD0A048261A5
:100D60007047816170474FF47A71B0FBF1F2521E07
:100D70004FF0E0235A6100229A6105221A6100BFF8
:100D8000704710B5044600F04FFB2060206800F06B
:100D900017FB6060606800F023FBA060606800F0F3
:100DA00031FBE06010BD00000248006800F03F0029
:100DB00070470000043802400248006800F48000D8
:100DC000704700000438024002480068C0F38810F1
:100DD000704700000438024030B50246012300BFCE
:100DE0001068C0F3801038BBD1E9000420438C6840
:100DF0002043CC6820430C6920434C6920438C6914
:100E00002043CC6920430C6A204314684FF6BF7519
:100E1000AC4320431060506820F004004C6940EA65
:100E200014405060086AB0F5005F04D1486A84B28B
:100E3000146100BF00BF0023D06920F40060D061BE
:100E4000184630BD014908607047000020000020AE
:100E50002DE9FF4104460D4601270026204600F0FB
:100E600075F8002859D1E96868680843296908437A
:100E7000A9690843E16849F20C6291430843E060C4
:100E8000A868216921F440510143216100BF6869CC
:100E9000616921F440710143616100BF6846FFF759
:100EA00070FF2048844201D1039E2BE01E488442FB
:100EB00001D1029E26E01D48844201D1029E21E01C
:100EC0001B48844201D1039E1CE01A48844201D190
:100ED000029E17E01848844201D1029E12E0174892
:100EE000844201D1029E0DE01548844201D1029E48
:100EF00008E01448844201D1039E03E01248844272
:100F000000D1039E4EB1286838B1002731462046F3
:100F10002B68AA6900F01FF800BF384604B0BDE88E
:100F2000F0810000001001400044004000480040F3
:100F300000140140004C0040005000400078004088
:100F4000007C004000180140001C01400146C868B8
:100F5000C0F3403070472DE9FC5F06460C469146D1
:100F60001D46B9F5004F68D10220A0FB057003466D
:100F70001920A4FB00A001463A465046FFF748F965
:100F80006421B0FBF1F04FEA001A0220A0FB0571CA
:100F90000B461920A4FB00B13A465846FFF738F932
:100FA00083460220A0FB057003461920A4FB000124
:100FB0003A46CDE90001FFF72BF96421B0FBF1F0CF
:100FC00000EBC00101EB0010ABEB8000322101EB24
:100FD000C0006421B0FBF1F000F0F8000AEB400A19
:100FE0000220A0FB057003461920A4FB00B13A467D
:100FF0005846FFF70DF983460220A0FB0570034613
:101000001920A4FB00013A46CDE90001FFF700F9E1
:101010006421B0FBF1F000EBC00101EB0010ABEB81
:101020008000322101EBC0006421B0FBF1F000F040
:101030000700504480B2B06067E00420A0FB057058
:1010400003461920A4FB00A001463A465046FFF78C
:10105000DFF882460420A0FB05711920A4FB00B034
:1010600084463A460B4658466146FFF7D1F864215C
:10107000B0FBF1F000EBC00101EB0010AAEB800027
:10108000322101EB00106421B0FBF1F000F0F00A16
:101090000420A0FB057003461920A4FB00B0014604
:1010A0003A465846FFF7B4F86421B0FBF1F00AEB7A
:1010B000001A0420A0FB057003461920A4FB00B110
:1010C0003A465846FFF7A4F883460420A0FB057073
:1010D00003461920A4FB00013A46CDE90001FFF7C1
:1010E00097F86421B0FBF1F000EBC00101EB0010B8
:1010F000ABEB8000322101EB00106421B0FBF1F07A
:1011000000F00F00504480B2B060BDE8FC9F0000CA
:1011100000B587B0182101A8FFF7D2F81020FFF71B
:101120005BFD0420FFF758FD8020FFF755FD0120EF
:10113000FFF752FD0220FFF74FFD0820FFF74CFD9F
:1011400010200104284A916100BF4FF6FF70019002
:10115000032002900020059001A92448FFF758FDC4
:101160004FF6EF700190032002900020059001A936
:101170001D48FFF74DFD03200190029000200590CF
:1011800001A91B48FFF744FD48F21F70019003209E
:1011900002900020059001A91648FFF739FD1020A4
:1011A000019001200290002003900490059001A975
:1011B0000D48FFF72DFD4FF2FF70019003200290C4
:1011C0000020059001A90C48FFF722FD4FF6FF70A3
:1011D0000190032002900020059001A90748FFF725
:1011E00017FD07B000BD00000008024000100240DB
:1011F000001C02400000024000040240000C0240BB
:1012000000B591B0282107A8FFF75AF8182101A8C6
:10121000FFF756F84FF48050FFF7ECFC0120FFF782
:10122000DBFCE020019002200290032003900020CC
:10123000049005900520069001A91248FFF7E8FCEC
:10124000002007904FF482700890002009900A90C7
:101250000B904FF400700C9008200D9000200E9021
:101260000F900A20109007A90748FFF7B5FD00204E
:101270000549496821F010010143034A516000BF4C
:1012800011B000BD000002400030014000B58DB03B
:101290001C2106A8FFF714F818216846FFF710F87C
:1012A0002020FFF7A7FC0120FFF796FC4FF4C05069
:1012B0000090022001900320029000200390012062
:1012C00004900820059069461448FFF7A1FC4FF4EC
:1012D000E130069000200790089009900C200A90B9
:1012E00000200B900C9006A90D48FFF7B1FD00BF40
:1012F0000B48006920F4904009490861084640699C
:1013000020F02A00486100BF00BF0846C06840F4D2
:101310000050C86000BF0DB000BD000000000240DA
:101320000014014000BFFEE7704770472DE9F0410F
:1013300005460C4617469846002624E0B85D144A38
:10134000216850542068401C2060701CC6B2288858
:1013500021880844C0F30A00A8B922680C4928680B
:10136000FFF7FCF922680A492868FFF7A5F920B9B8
:10137000226808A0296800F009FC28682168084450
:101380002860002020604645D8DBBDE8F0810000E1
:10139000280000202A2A2A2056657269667920666C
:1013A0006C617368206661696C65642061742025D6
:1013B0003038582C2025642062797465730D0A003A
:1013C000014600BF0448006800F0F0000009034A2D
:1013D000125C21FA02F0704708380240C823000866
:1013E000014600BF0548006800F4E050044A02EBE3
:1013F0009020027821FA02F070470000083802407D
:10140000D8230008014600BF0548006800F460408A
:10141000044A02EB5030027821FA02F070470000D3
:1014200008380240D823000810B5002400BF0C483B
:10143000006800F00C0020B1042804D0082809D16D
:1014400003E0084C08E0084C06E0082000F00EF825
:10145000044601E0034C00BF00BF204610BD000061
:10146000083802400024F40040787D012DE9F04165
:101470000446002500260027FFF79EFC06461EB105
:10148000B6F5800F04D101E00E4D03E00E4D01E0F2
:101490000C4D00BF00BF082C11D1FFF785FCB5FB38
:1014A000F0F8FFF791FC08FB00F80848006800F42A
:1014B0004030012101EB10404000B8FBF0F7384606
:1014C000BDE8F0810024F40040787D01043802403A
:1014D0002DE9F04105460E46174600F067FB8046B1
:1014E00072B610212948FFF739FC032028490873F8
:1014F00000BF2748806800F001000028F9D0244888
:10150000007B280C2249087300BF2148806800F046
:1015100001000028F9D01E48007B280A1C490873E6
:1015200000BF1B48806800F001000028F9D018486F
:10153000007B17490D7300BF1548806800F001005B
:101540000028F9D01248007B00240DE0002010494B
:10155000087300BF0E48806800F001000028F9D031
:101560000B48007B3055641CBC4203D22819B0F5EF
:10157000000FEBD310210548FFF7F3FBB8F1000F84
:1015800000D162B62046BDE8F081000000080240AC
:10159000003001402DE9F04106460F46144617E0A1
:1015A000B4F5807F02D94FF4807500E025462A46C5
:1015B00009493046FFF78CFF2A4639460648FEF7B0
:1015C0008AFE10B10020BDE8F0812E442F44641B38
:1015D000002CE5D10120F6E73C0800202DE9F0477A
:1015E0000646884615462848007838B10020264926
:1015F0000870FF22511C2548FEF75BFE3FE0F4B265
:10160000C4F58077AF4200D92F46361B4FF4807265
:101610001F493046FFF75CFF1D4908193A4641460D
:10162000FEF759FE38B31A4908193A461749FEF72A
:1016300052FE60B100F0BAFA814672B600F088F945
:10164000304600F035F8B9F1000F00D162B610490C
:1016500008193A464146FEF70CFE00F0A7FA81460B
:1016600072B600F075F90A49304600F085F8B9F114
:10167000000F00D162B606F58076B844ED1B002D50
:10168000BDD10120BDE8F087110000203C0A0020F8
:101690003C08002010B500BF0448006840F040003E
:1016A0000249086000BF00F0E5F810BD00300140BD
:1016B00070B50446FF2510212D48FFF74FFB812010
:1016C0002C49087300BF2B48806800F001000028F7
:1016D000F9D02848007B200C2649087300BF254814
:1016E000806800F001000028F9D02248007B200A21
:1016F0002049087300BF1F48806800F001000028DF
:10170000F9D01C48007B1B490C7300BF1948806846
:1017100000F001000028F9D01648007B1021144881
:10172000FFF71FFB00BF10211148FFF717FB052033
:101730001049087300BF0F48806800F001000028BE
:10174000F9D00C48007B00200A49087300BF094803
:10175000806800F001000028F9D00648057B1021C0
:101760000348FFF7FEFA05F001000028DBD170BD49
:1017700000080240003001402DE9F04105460E46C8
:10178000FF2710213948FFF7E9FA0220384908738A
:1017900000BF3748806800F001000028F9D03448C5
:1017A000007B280C3249087300BF3148806800F084
:1017B00001000028F9D02E48007B280A2C49087324
:1017C00000BF2B48806800F001000028F9D02848AD
:1017D000007B27490D7300BF2548806800F0010099
:1017E0000028F9D02248007B00240DE0305D20491C
:1017F000087300BF1E48806800F001000028F9D07F
:101800001B48007B601C84B2FF2C03DC2819B0F558
:10181000000FEBD310211548FFF7A3FA00BF1021EA
:101820001248FFF79BFA05201149087300BF1048C2
:10183000806800F001000028F9D00D48007B0020EE
:101840000B49087300BF0A48806800F001000028B7
:10185000F9D00748077B10210448FFF782FA07F008
:1018600001000028DBD12046BDE8F08100080240DD
:101870000030014070B500F099F9054672B61021AC
:101880001848FFF76BFA9F201749087300BF1648E6
:10189000806800F001000028F9D01348007B13A0F5
:1018A00000F074F9002410E000200F49087300BF15
:1018B0000D48806800F001000028F9D00A48017B3B
:1018C0000EA000F063F9601CC4B2032CECDB0DA089
:1018D00000F05CF910210348FFF743FA05B962B63E
:1018E00070BD000000080240003001400D0A466C47
:1018F0006173682049442069733A200025303258CA
:10190000200000000D0A000010B500F04FF9044659
:1019100072B600F01DF810210B48FFF71FFA98204F
:101920000A49087300BF0948806800F001000028D8
:10193000F9D00648007B10210348FFF712FA04B9DA
:1019400062B6012010BD00000008024000300140D6
:1019500010B5002410211E48FFF700FA06201D498B
:10196000087300BF1B48806800F001000028F9D010
:101970001848007B10211648FFF7F3F9102114488E
:10198000FFF7ECF905201349087300BF1148806880
:1019900000F001000028F9D00E48007B00200D491E
:1019A000087300BF0B48806800F001000028F9D0E0
:1019B0000848047B10210648FFF7D3F904F0020021
:1019C00008B1012010BD04A000F0E0F80020F9E704
:1019D00000080240003001400D0A5772697465200A
:1019E000656E61626C65206661696C65640D0A00F4
:1019F0007047000070B502205749096821F00F01B7
:101A00000143554A116000BF00BF1046006800F056
:101A10000F00022801D0FEF7A0FC4FF440404F49D0
:101A2000096821F4404101434C4A116000BF102075
:101A30004B49096821F0F80141EAC001484A1160A8
:101A400000BF00BF1046006840F00100114608606A
:101A500000BF00BF00BF42480068C0F3400000283C
:101A6000F8D0002008214022034640EA010444EA5D
:101A700082143B4D2D1D2D683A4E35402C43384D78
:101A80002D1D2C602C46246824F440341C432C600B
:101A900000BF00BF281F006840F08070291F086049
:101AA00000BF00BF00BF2E480068C0F340600028A0
:101AB000F8D000202A490831096821F0F0010143DB
:101AC000274A0832116000BF90141146096821F4BA
:101AD000E0510143116000BF00201146096821F464
:101AE00060410143116000BF02201146096821F0E6
:101AF00003010143116000BF00BF00BF1848083058
:101B0000006800F00C000828F7D11748FFF72BF900
:101B10000420042808D14FF0E021096941F00401B4
:101B20004FF0E022116107E04FF0E021096921F058
:101B300004014FF0E022116100BF0B48FFF782F96A
:101B4000002007498C31096821F080710143044A63
:101B50008C32116000BF70BD003C0240007000403C
:101B6000003802400080BFFF0090D00305480068A5
:101B700040F47000034908604FF00060014980396B
:101B80000860704788ED00E000BFFEE70FB4054B2A
:101B900010B503A9044A029800F01AF810BC5DF8C9
:101BA00014FB0000E121000824000020EFF3108066
:101BB000704702E008C8121F08C1002AFAD1704716
:101BC0007047002001E001C1121F002AFBD17047BD
:101BD0002DE9FF4F8DB00F460546002606E025286B
:101BE0000BD0DDE90F1290476D1C761C2878002879
:101BF000F5D111B03046BDE8F08F0024A246A146D1
:101C00000122EC4900E0044315F8013F203B02FAB1
:101C100003F00842F7D128782A2810D06FF02F025D
:101C20002878A0F13001092914D80AEB8A0102EBC7
:101C3000410144F0020400EB010A6D1CF0E701CF02
:101C40005FEA000A03D544F40054CAF1000A44F0E4
:101C500002046D1C28782E2817D115F8010F44F0C6
:101C600004042A280ED06FF02F022878A0F130014A
:101C700009290AD809EB890102EB410100EB0109AE
:101C80006D1CF2E757F8049B6D1C28786C280FD068
:101C900006DC4C2817D068280DD06A2814D104E03F
:101CA000742810D07A280FD10DE044F400140AE013
:101CB00044F4801401E044F440146978814202D174
:101CC00004F580146D1C6D1C2A786E2A1FD00CDC64
:101CD000632A31D004DC002A8BD0582A11D1A3E02A
:101CE000642A68D0692A0CD165E0732A2ED004DCFE
:101CF0006F2A73D0702A04D19BE0752A6FD0782A9E
:101D00006ED01046DDE90F129047761C50E1C4F307
:101D10000250022806D0032809D0042801CF09D098
:101D2000066045E101CFF117C0E9006140E101CF54
:101D300006803DE106703BE117F8040B8DF80000CA
:101D400000208DF80100EB46012003E057F804BBAA
:101D50004FF0FF3061074FF0000102D40DE008F1B1
:101D60000101884649450FDA8045F8DB1BF8081069
:101D70000029F4D108E008F1010188468142FADB2C
:101D80001BF808100029F6D1DDE90F23AAEB0800A3
:101D90008146214600F036F9304400EB080604E0A5
:101DA000DDE90F121BF8010B9047B8F10108F7D2DB
:101DB00021464846F7E00A21C4F302534FF0000BD6
:101DC0000891022B04D001CFC117032B09D00AE0E0
:101DD000FF1D27F00707F7E8020108E032E01FE0E7
:101DE00020E000B2C117042B01D140B2C117031E7D
:101DF00071F1000307DA4FF0000CD0EB0C006CEB34
:101E000001012D2302E0230504D52B238DF8243076
:101E1000012303E0E30701D02023F7E7984658E0C9
:101E20000A2110E010210EE010204FF0000B089066
:101E30000CE010214FF0000B44F004044FF00809AF
:101E4000089103E008214FF0000B0891C4F30253FE
:101E5000022B04D001CF0021032B06D006E0FF1D8A
:101E600027F00707F7E8020103E080B2042B00D156
:101E7000C0B24FF0000823072BD5702A07D0DDF839
:101E800020C08CF0100C5CEA0B0C05D00EE0402357
:101E90008DF82430012308E050EA010306D03023F6
:101EA0008DF824308DF8252002239846DDF820C0D7
:101EB0008CF0080C5CEA0B0C0BD150EA010301D149
:101EC000630706D530238DF824304FF00108A9F1BF
:101ED0000109582A04D038A20B9208AA0A920BE0F2
:101EE0003AA2F9E75B46089AFEF792F90B9B9B5CD6
:101EF0000A9A521E0A92137050EA0102F2D10A980D
:101F0000ADEB000000F1200B600702D524F4803413
:101F100001E04FF00109D94502DDA9EB0B0000E01B
:101F2000002000EB0B0141440890AAEB010AE003FA
:101F300006D4DDE90F232146504600F063F806443D
:101F40004FF0000908E009A911F80900DDE90F12B6
:101F5000904709F10109761CC145F4DBE0030CD57B
:101F6000DDE90F232146504600F04CF8064404E01A
:101F7000DDE90F1230209047761C0899481E089022
:101F80000029F5DC08E00A980A990078491C0A91B2
:101F9000DDE90F129047761CBBF10001ABF1010B9C
:101FA000F1DC21465046DDE90F2300F019F8064424
:101FB0006D1C1BE6092801003031323334353637C9
:101FC0003839616263646566000000003031323385
:101FD0003435363738394142434445460000000025
:101FE0002DE9F041044600251E461746880404D416
:101FF00005E039462020B0476D1C641EF9D52846FF
:10200000BDE8F0812DE9F041044600251E469046CA
:10201000C80301D5302700E02027880404D505E057
:1020200041463846B0476D1C641EF9D52846BDE8C8
:10203000F08100002DE9F04188B006460F46904639
:102040000020079006900590019657E0012306AA0C
:1020500007A93846FEF798FC012840D10C2306AAB0
:1020600007A93846FEF790FC441C032306AA07A9DB
:102070003846FEF789FCC01CC5B20598844208DCCE
:102080002C48059A1044011B2A4602A8FEF7F1F8D5
:102090001EE00598201AA84208DB0599611A019AEA
:1020A000501A2A4602A9FEF7BFFA11E00599621AF2
:1020B000611A019B581A02A9FEF7B6FA0599611A2E
:1020C0006A1A0599611A02ABC8181A49FEF7D1F8C5
:1020D0002B4602AA05A901A8FFF728F90EE008235C
:1020E00006AA07A93846FEF74FFCC0B28DF80800D3
:1020F000012302AA05A901A8FFF718F9A8F1010018
:1021000007998842A2DC059800280FDD0949059A45
:102110000198FEF723FB0749059A0198FEF7CCFAD0
:1021200020B905A0059A0199FFF730FD08B0BDE878
:10213000F0810000280000202A2A2A2056657269B2
:10214000667920666C617368206661696C656420DD
:10215000617420253038582C2025642062797465FC
:10216000730D0A0070B50B46002114E05C5C00257D
:102170000DE080EA040606F0010626B14AF20106E7
:1021800086EA600000E0401064106E1C35B2082D35
:10219000EFDB4E1C31B29142E8DB70BD2DE9F0411E
:1021A00006460C46002713E0B4F5807F02DD4FF4AD
:1021B000807500E0A5B22A4608493046FFF788F945
:1021C0002AB206493846FFF7CDFF07462E44641B66
:1021D000002CE9DC3846BDE8F08100003C09002015
:1021E00070B505460C460548844203D1284600F0E8
:1021F000DDF870BD4FF0FF30FBE700002400002049
:1022000008B54FF48040FEF7F5FC4FF080501349BD
:1022100009680143114A11601146096801400091A3
:1022200000BF00BF032002460D4B19684FF6FF03A5
:1022300019400C4B0B4343EA0221094B196000BFC4
:10224000FFF7D8FBFEF764FFFEF7DAFFFFF71EF893
:10225000002000F009F800BFFEE70000403802400F
:102260000CED00E00000FA050EB500200090019092
:102270000290FFF70FFA0C2269464FF48020FFF717
:1022800027F9BDF8000045F2AA51884245D19DF8D2
:10229000020000F0010000283FD00C226946002017
:1022A000FFF760FF002838D122480199FFF776FF39
:1022B000002832D120A0FFF769FCFEF753FC9DF8FF
:1022C0000200800930B90198821E1A492348FEF79E
:1022D00075FA05E00198821E16492048FFF7AAFE0C
:1022E000FEF7EAFBFFF710FB9DF8020020F001006B
:1022F0008DF802000C2269464FF48020FFF76EF93A
:102300000C2269464FF48020FFF744F928B90C22CB
:102310004FF4802112A0FFF739FC1DA0FFF736FC17
:1023200000BF2148006800F040000028F9D00B48A9
:10233000FEF73AFC0C0004000D0A4465636F6D70F3
:102340007265737320757067726164652070616374
:102350006B616765202E2E2E0D0A000000400008DC
:102360002A2A2A205665726966792053466C617361
:1023700068206661696C6564206174202530385876
:102380002C2025642062797465730D0A000000001A
:102390000D0A4A756D7020746F204150524F4D20C8
:1023A0002E2E2E0D0A0000000014014000BF05492A
:1023B000096801F080010029F9D0C1B2014A121D5B
:1023C0001160704700140140000000000000000090
:1023D00001020304060708090000000001020304CB
:1023E000002400080000002028000000B21B0008A4
:1023F0002824000828000020380F0000C21B000815
:1024000001000000000000000000000000000000CB
:1024100000010000000000001000000001000000AA
:082420000090D0030000000051
:04000005080001D915
:00000001FF
